:100000000C941E060C94F6270C9423280C94460698
:100010000C9446060C9446060C9446060C94460630
:100020000C9446060C9446060C942C130C9446062D
:100030000C9446060C9446060C9446060C94460610
:100040000C9450280C9446060C943E2C0C94812C55
:100050000C9446060C9446060C9446060C944606F0
:100060000C9446060C9446068F18F118D018D31835
:10007000D618D918DC18DF18E218F118EB18231A73
:10008000251A251A231A251A251A251A251A251A7A
:10009000251A251A251A251A251A251A251A251A68
:1000A000A919251A251A251A251A251A1A19251AE1
:1000B000251A251A251A251A251A251A251A251A48
:1000C000251A251A251A251A251A251AB519B5191A
:1000D000B519B519B519B519B519B519B519251A3F
:1000E000251A251A251A251A251A1A19B419B41908
:1000F000B419B419251AC219C819CE19D419DA19A4
:10010000E019E619EC19F619001A0A1A141A5B1903
:100110001D19251A251A251A251AA919251A251A6D
:10012000251A251A251A251A251A251AB319B319BD
:10013000B319B319251AC219C819CE19D419DA1965
:10014000E019E619EC19F619001A0A1A141A5B19C3
:100150001D19251A251A251A251AA919581A581AC7
:10016000581A581A581A581A581A581A581A581AFF
:10017000581A581A581A6E1B6E1B6E1B6E1B6E1B7C
:100180006E1B9D1AA71AB11ABB1A181B221B311B12
:10019000421BCA1CDF1CEB1CF41C031D281D311D57
:1001A0007A1D431D8D2093209920A020AE20D020C1
:1001B000EE20456E746572206D656E752E2E2E00D4
:1001C000546F67676C6564206D6963726F50504D42
:1001D00000546F67676C656420696E76657274653C
:1001E000642050504D2100546F67676C6564205443
:1001F00058206D7574696E672100546F67676C6570
:10020000642074656C656D65747279210050726F3D
:10021000746F636F6C206572726F72207769746897
:100220002052580054696D656F7574207768656E4B
:1002300020636F6E6E656374696E6720746F205201
:100240005800507265737320616E79206B65792058
:10025000746F2063616E63656C00436F6E6E6563DF
:1002600074696E6720746F2052582C20706F776508
:100270007220757020746865205258202877697440
:10028000682062696E6420706C7567206966206EF4
:100290006F74207573696E6720616C776179732064
:1002A00062696E642900546F67676C656420276912
:1002B0006D6D656469617465206F75747075742700
:1002C00000546F67676C65642027736C61766520E6
:1002D0006D6F64652700546F67676C6564202761E4
:1002E0006C776179732062696E642700546F676769
:1002F0006C65642050504D206368616E6E656C20A3
:100300006C696D69740053657420525353492069B8
:100310006E6A656374696F6E206368616E6E656C8A
:100320002028303D3D64697361626C652900536526
:10033000742050504D206D696E696D756D20737914
:100340006E630053657420626561636F6E20696E31
:1003500074657276616C0053657420626561636FC9
:100360006E2064656C617900536574206265616319
:100370006F6E206672657175656E637920696E2097
:10038000487A3A20303D64697361626C652C205074
:10039000783D504D52206368616E6E656C20782CFC
:1003A0002046783D465253206368616E6E656C202E
:1003B00078005365742050574D2073746F7020641B
:1003C000656C61792028302064697361626C6564B2
:1003D0002C20312D323535203D3D20302E317320FB
:1003E0002D2035306D696E29005365742050504DB5
:1003F0002073746F702064656C61792028302064EC
:10040000697361626C65642C20312D323535203D75
:100410003D20302E3173202D2035306D696E29003E
:10042000536574206661696C736166652064656CF0
:1004300061792028302064697361626C65642C20C6
:10044000312D323535203D3D20302E3173202D2089
:1004500035306D696E29002A2A2A2A2A2A2A2A2A50
:100460002A2A2A2A2A2A2A2A2A2A2A2A2A2A2A2AEC
:100470002A2A2A2A0052582041636B6564202D20C5
:1004800072657665727420737563636573736675E0
:100490006C21002A2A2A2A2A2A2A2A2A2A2A2A2AAD
:1004A0002A2A2A2A2A2A2A2A2A2A2A2A2A2A2A2AAC
:1004B000002A2A2A2A2A2A2A2A2A2A2A2A2A2A2AC6
:1004C0002A2A2A2A2A2A2A2A2A2A2A2A2A2A00528E
:1004D000582041636B6564202D20757064617465DC
:1004E000207375636365737366756C21002A2A2A0D
:1004F0002A2A2A2A2A2A2A2A2A2A2A2A2A2A2A2A5C
:100500002A2A2A2A2A2A2A2A2A2A0056616C696457
:100510002063686F69636573206172653A205B319F
:100520005D2D5B31365D20286368616E6E656C20E1
:10053000312D31362900536574206F7574707574D0
:1005400020666F7220706F727420005B585D2061AE
:10055000626F7274206368616E67657320616E6498
:10056000206578697420525820636F6E6669670051
:100570005B535D20736176652073657474696E6783
:100580007320746F205258005B525D20726576654F
:1005900072742052582073657474696E6773207486
:1005A0006F2064656661756C747300557365206EA9
:1005B000756D62657273205B312D445D20746F2010
:1005C0006564697420706F727473205B452D515D92
:1005D00020666F722073657474696E677300202DD6
:1005E00020726563656976657220636F6E66696700
:1005F000757261746F722C20727820737720000AF4
:100600000A6F70656E4C52536E67200053657420FC
:1006100073657269616C2062617564726174653AB8
:10062000200056616C69642063686F696365733A82
:100630002031202D20342B34202F2032202D203823
:10064000202F2033202D20382B34202F2034202D14
:10065000203132202F2035202D2031322B34202FF5
:100660002036202D20313600536574204368616E9A
:100670006E656C20636F6E6669673A20005365741F
:100680002044617461726174652028302D32293AEA
:10069000200053657420486F70206368616E6E653A
:1006A0006C7320286D61782032342C207365706162
:1006B000726174656420627920636F6D6D61732966
:1006C0002076616C69642076616C75657320312DCC
:1006D0003235353A2000536574206368616E6E656B
:1006E0006C2073706163696E6720287831306B48C5
:1006F0007A293A200053657420524620706F77653E
:10070000722028302D37293A200053657420524634
:10071000206D6167696320286865782920652E67E8
:100720002E20307844454144463030443A2000532E
:1007300065742062617365206672657175656E63AC
:10074000792028696E20487A293A20005B5A5D207A
:10075000656E746572207265636569766572206383
:100760006F6E66696775726174696F6E2075746902
:100770006C79005B465D20646973706C61792061FF
:10078000637475616C206672657175656E63696509
:10079000732075736564005B525D2063616C6375E3
:1007A0006C6174652072616E646F6D206B65792079
:1007B000616E6420686F70206C697374005B495DC2
:1007C000207265696E697469616C697A6520736508
:1007D0007474696E677320746F20736B65746368DB
:1007E0002064656661756C7473005B585D2072658A
:1007F00076657274206368616E67657320616E64EC
:100800002065786974206D656E75005B535D20739B
:100810006176652073657474696E677320746F20E8
:10082000454550524F4D20616E64206578697420B3
:100830006D656E7500557365206E756D62657273BA
:10084000205B302D395D20746F20656469742070E1
:100850006172616D657465727300202D2053797328
:1008600074656D20636F6E66696775726174696F18
:100870006E000A0A6F70656E4C52536E672000510D
:1008800029204F7574707574206265666F726520DB
:100890006C696E6B20283D465329203A2000502970
:1008A00020536C617665206D6F64652028657870D3
:1008B0006572696D656E74616C293A20004F29205C
:1008C00054696D65642042494E44206174207374FC
:1008D000617274757020203A20004E292050504DCE
:1008E000206F7574707574206C696D69746564200F
:1008F000202020203A200044495341424C454400E6
:100900004D292050504D205253534920746F20637D
:1009100068616E6E656C202020203A20004C2920F2
:1009200050504D206D696E696D756D2073796E63E1
:10093000202875732920203A200044495341424C15
:100940004544004B29204661696C736166652062ED
:100950006561636F6E20696E74762E2028312D32AA
:10096000353573293A20004A29204661696C736144
:10097000666520626561636F6E2064656C617920D5
:1009800028302D323535203D3E20313073202D204A
:100990003135306D696E293A200049292046616958
:1009A0006C7361666520626561636F6E206672714B
:1009B0002E203A200048292050574D2073746F7024
:1009C0002064656C6179202020202020203A2000BE
:1009D00047292050504D2073746F702064656C61FE
:1009E00079202020202020203A200046292046611E
:1009F000696C736166652064656C617920202020D4
:100A00002020203A200050574D206368616E6E65AB
:100A10006C200066756E6374696F6E3A2000292041
:100A2000706F72742000506F776572546F776572C3
:100A300000445446205548462033322D62697420C4
:100A400031306368004F70656E4C52536E67525878
:100A5000206D696E6920342F36636800466C7974A6
:100A6000726F6E2F4F72616E6765525820554846FF
:100A70002038636800525820747970653A20004429
:100A8000697361626C656400487A00203D3D200016
:100A900043616C63756C61746564207061636B6540
:100AA0007420696E74657276616C3A200042292068
:100AB0004D6963726F202868616C66292050504D23
:100AC000202020203A00412920496E766572746505
:100AD000642050504D20696E20202020203A0030A4
:100AE00029204D7574652062757A7A657220286DAB
:100AF0006F73746C79293A003929205365726961E2
:100B00006C2062617564726174653A00736D617224
:100B100074506F7274004672536B79005472616E38
:100B200073706172656E740044697361626C6564B0
:100B30000038292054656C656D657472793A2020FF
:100B40002020202020003729204368616E6E656CCC
:100B500020636F6E6669673A202000362920446161
:100B60007461726174652028302D32293A2020206A
:100B700000352920486F70206368616E6E656C7364
:100B80003A2020202020003429204368616E6E65C1
:100B90006C2073706163696E673A202000332920EE
:100BA000524620706F7765722028302D37293A2001
:100BB0002020003229205246206D616769633A2067
:100BC0002020202020202020003129204261736530
:100BD000206672657175656E63793A202020000089
:100BE00000000700020100000304060000000000EE
:100BF00000000001020408102040800102040810D7
:100C00002001020408102004040404040404040263
:100C10000202020202030303030303000000002395
:100C2000002600290000000000250028002B0000FD
:100C3000000000240027002A00006F2D11241FBE91
:100C4000CFEFD8E0DEBFCDBF13E0A0E0B1E0ECEE27
:100C5000F0E602C005900D92A83CB107D9F716E066
:100C6000A8ECB3E001C01D92AE38B107E1F71CE07B
:100C7000CCE3DCE004C02297FE010E94782ECA3348
:100C8000D107C9F70E94AB2D0C9474300C9400006E
:100C900080917305813019F482E08093730580910F
:100CA0007305833019F484E0809373050895A89543
:100CB0000895DC01ED91FC910190F081E02D099502
:100CC00008952091740530917505382748E0C901D1
:100CD000880F991F37FF06C09C0151E2252750E17C
:100CE000352701C09C01415091F730937505209341
:100CF0007405089588E38093760580E092ECA1E086
:100D0000B0E08093770590937805A0937905B09330
:100D10007A0587E08093830580E091EAACEBB3E34A
:100D200080937B0590937C05A0937D05B0937E0511
:100D300085E0809384058DEE9EEFADEABEED809355
:100D40007F0590938005A0938105B0938205E5E827
:100D5000F5E080E090E0863028F4DC01AE54BC4F32
:100D60002C9101C020E0219301968831910599F7DB
:100D700082E080939D058AE080939E05089580E03F
:100D80009EECADEEB4E38093BB059093BC05A093BD
:100D9000BD05B093BE0580E090E0A0E0B0E5809393
:100DA000BF059093C005A093C105B093C205E3ECC5
:100DB000F5E080E081938F5F8031E1F70895A0E056
:100DC000B0E0E5EEF6E00C94412ED82F0E94A62864
:100DD0006115710581059105C9F30E94E42E1092F9
:100DE0007F05109280051092810510928205C4E063
:100DF000812C912C54018A94C0907F05D09080055D
:100E0000E0908105F0908205FE2CED2CDC2CCC24AA
:100E10000E94DF2EA50194010E94202E6C0D7D1DE5
:100E20008E1D9F1D60937F057093800580938105C3
:100E300090938205C15001F7DD2309F450C005E805
:100E400015E0E801A12CB12C62E3C62ED12CE12CD7
:100E5000F12C8881882309F442C0B39419F40E94CC
:100E60007A063DC00E94DF2EA70196010E94202E27
:100E7000E1E0E60FA5E8B5E08A2F801B8A1520F493
:100E80008D918E13F9CFE9CF2091840530E0A0E158
:100E9000B7E20E94B82D9B01AC01AE2FB0E00E94DA
:100EA000C72D40907B0550907C0560907D0570902B
:100EB0007E05640D751D861D971D4090BB055090E5
:100EC000BC056090BD057090BE05461657066806C5
:100ED000790618F2E993A39488E1A812BACFCDB7A6
:100EE000DEB7E0E10C945D2E8436910520F4BC0160
:100EF00080E090E017C09C018E3B910528F42A55B4
:100F00003109AAE0B0E00CC0823D910528F4245BD1
:100F10003109A4E6B0E004C02D5C3109A8E5B2E0D7
:100F20000E94B82DA4E6B0E09B01AC010E94C72D41
:100F3000089590E08C599F4F0E947407089561E0D6
:100F400083E10E94532960E083E10E948C2982E0C2
:100F50008093B00085E08093B10061E083E00E945F
:100F6000532960E083E00E948C290895A4E0B0E05A
:100F7000ECEBF7E00C944F2E009749F19C0140E018
:100F800050E068E478EE81E090E00E94202E61E07D
:100F900083E129833A834B835C830E948C292981D6
:100FA000822F3A81932F4B81A42F5C81B52F8F3FE5
:100FB0009105A105B10529F020F08FEF90E0A0E0A8
:100FC000B0E08093B3008091B000806107C060E022
:100FD00083E10E948C298091B0008F7E8093B000C5
:100FE0002496E2E00C946B2E60E08CE00E94532982
:100FF00061E08BE00E94532961E08DE00E9453295B
:1010000060E082E00E94532961E084E00E9453295D
:10101000089542E050E068E476E080E00E94D62740
:101020000895E3E0F0E089E080935700E491E670F2
:1010300081E0E63009F080E00895CF93DF93C82F78
:101040000E941108882381F0DFB781E08093720548
:10105000F8940E94570688E180936000C093600076
:10106000C1110E945706DFBFDF91CF9108958F9283
:101070009F92AF92BF92CF92DF92EF92FF92CF9367
:10108000FC01C0A5EC2FE770F0E0E658FC4FA08112
:10109000B0E0C7FF03C024E130E002C02FE030E041
:1010A000FC0197A183E1989FF0011124E25CFE4FBF
:1010B00080809180A280B380A20FB31F20E43FE123
:1010C0004DE750E00E94D22DA50194010E94FE2D13
:1010D0008C2F887149F469017A01E0EDCE0EE7E0CA
:1010E000DE1EE11CF11C1BC0C7FF05C060E47AE8EE
:1010F0008CE29EE004C060E07EEE8AEB9BE069013A
:101100007A01F8EBCF0EFBE0DF1EE11CF11CA5011C
:1011100094010E94FE2DC20ED31EE41EF51EC701CF
:10112000B60169517C4F8F4F9F4F28EE33E040E06E
:1011300050E00E94FE2DA8EEB3E00E94C72DCF9193
:10114000FF90EF90DF90CF90BF90AF909F908F90E7
:1011500008958F3F910551F048F0811522E09207E4
:1011600038F08115934030F482E0089580E00895CE
:1011700081E0089583E00895A0E0B0E0E2ECF8E0BB
:101180000C944A2EEB018A01B82FB695A0E0288175
:101190003981F80120832A813B8121832C813D8183
:1011A00022832E813F812383688179814A815B81FB
:1011B0002C813D81EE81FF819F2F9295990F990F90
:1011C000907C272F2370922B252F2370220F220F24
:1011D000922B232F23702295207F922BF80194834A
:1011E0000B5F1F4F2896AF5FBA1788F680FF24C0A9
:1011F000888199810E94A908D82E8A819B810E94AA
:10120000A908E82E8C819D810E94A908F82E8E8164
:101210009F810E94A908F0E4DF9EA001112490E1C3
:10122000E99E90011124242B282BE4E0FE9EB001BE
:101230001124262BF8012083CDB7DEB7E7E00C940C
:10124000662E803223E0920708F1883E23E0920761
:1012500040F48F519340E4E096958795EA95E1F745
:101260000895803D27E0920718F48C5D934008951F
:10127000883928E0920768F4885C974074E0969576
:1012800087957A95E1F78D509C4F089580E090E026
:1012900008958FEF93E008958C30910540F4A4E019
:1012A000880F991FAA95E1F7885D9C4F0895843FA8
:1012B00023E0920718F484529C4F0895811524E08E
:1012C000920740F48657934FF4E0880F991FFA95E0
:1012D000E1F7089580E998E008959C0136952795F7
:1012E00025753575821B930B9C012373337396957B
:1012F00087959695879583739373820F931F9C01AF
:1013000054E0369527955A95E1F7280F391F2F702D
:101310003F7041E051E0249FC001259F900D349F14
:10132000900D1124892F08952D98882319F000001D
:101330002B9A02C000002B9800002D9A00000895FF
:101340002D9A000083B12D98000082958170089538
:10135000CF93DF93D82F5C9A2D985C98C8E08D2F9F
:1013600080780E949409DD0FC150C9F72D98DF9154
:10137000CF9108958F770E94A8090895CF93DF93A6
:10138000D82FC8E08D2F80780E949409DD0FC150BE
:10139000C9F72D98DF91CF910895CF93DF932D98C2
:1013A000C8E080E0D82FDD0F0E94A0098D0FC1504A
:1013B000C9F7DF91CF9108950E94BA090E94CD0923
:1013C0005C9A0895A1E0B0E0E8EEF9E00C944F2EAD
:1013D000806869830E94A8096981862F0E94BE09DE
:1013E0005C9A2196E2E00C946B2ECF93C0917F051E
:1013F000C827E82FF0E0EA58FA4F678589E70E948E
:10140000E2096C2F8DE30E94E2096C2F82E40E94B6
:10141000E209CF91089586E20E94DC090895CF93F6
:10142000DF93EC016C818CE10E94E2096D818DE11A
:101430000E94E2096E818EE10E94E2096F8180E2E2
:101440000E94E209688581E20E94E209698582E2E0
:101450000E94E2096A8583E20E94E2096B8584E2C8
:101460000E94E2096C8585E20E94E2096D858AE2AC
:101470000E94E2096E858EE60E94E2096F858FE682
:101480000E94E209688980E70E94E209698981E790
:101490000E94E2096A8982E70E94E209DF91CF9106
:1014A0000895CF92DF92EF92FF92CF93DF936B017B
:1014B0007C01C11488E3D8068CE9E8068CE1F806C3
:1014C00028F5C701B60120E836E948E950E00E9456
:1014D000FE2DE901689760E879E687E69FEF0E94B4
:1014E000DA2D6C0D7D1D8E1D9F1DF2E0660F771F9E
:1014F000881F991FFA95D1F721E732E040E050E0CC
:101500000E94FE2DF22EE32E80E421C0C701B60119
:1015100020E03DE241E351E00E94FE2DE9016897A1
:1015200060E073ED8EEC9EEF0E94DA2D6C0D7D1D58
:101530008E1D9F1D660F771F881F991F21E732E0C0
:1015400040E050E00E94FE2DF22EE32E80E66C2F4C
:101550006F71680F85E70E94E2096E2D86E70E9491
:10156000E2096F2D87E70E94E209DF91CF91FF909A
:10157000EF90DF90CF900895682F8DE60E94E209EA
:1015800008958F929F92AF92BF92CF92DF92EF9287
:10159000FF92CF93DF93D82F83E00E94DC098093E2
:1015A000710584E00E94DC098093700560E086E0AC
:1015B0000E94E20961E087E00E94E2096FE789E0AA
:1015C0000E94E20965E08AE00E94E20962E18BE0A4
:1015D0000E94E20965E18CE00E94E2096DEF8DE076
:1015E0000E94E20960E08EE00E94E209DD2319F02A
:1015F0008BE291E008C020919D0533E1239FC0015B
:101600001124825C9E4F0E940F0A6CE880E30E94C6
:10161000E2096FE082E30E94E20962E483E30E9450
:10162000E20980919E0587FF02C064E101C06AE083
:1016300084E30E94E2096AE285E30E94E2096DE226
:1016400086E30E94E20964ED87E30E94E20960E01C
:1016500088E30E94E20960E089E30E94E209D11177
:1016600009C0C0907F05D0908005E0908105F09082
:10167000820507C0C5E9CC2EC1ECDC2EED2CCEEDE9
:10168000FC2ECAE38F2C9924AA24BB24682D8C2F0E
:101690000E94E209682D85E08C0F0E94E209FE2C71
:1016A000ED2CDC2CCC24CF5FCE3361F76FEF83E4DD
:1016B0000E94E2096FEF84E40E94E2096FEF85E483
:1016C0000E94E2096FEF86E40E94E209DD2311F037
:1016D00066E002C0609183058DE60E94E20960E049
:1016E00089E70E94E209609184058AE70E94E20985
:1016F00060E083E70E94E20960E084E70E94E2097B
:10170000D11109C060917B0570917C0580917D05A8
:1017100090917E0504C060E071EA8CEB93E30E9437
:10172000510ADF91CF91FF90EF90DF90CF90BF9063
:10173000AF909F908F90089561E087E00E94E2094A
:1017400064E28EE70E94E20963E088E00E94E20919
:1017500060E088E00E94E20965E087E00E94E2091B
:1017600062E085E00E94E20983E00E94DC09809348
:10177000710584E00E94DC0980937005089583E080
:101780000E94DC098093710584E00E94DC0980934B
:10179000700561E087E00E94E2096AE070E080E0A5
:1017A00090E00E94C9280E949C0B00000895CF92EF
:1017B000DF92FF920F931F93CF93DF931F92CDB7CA
:1017C000DEB7082F162F8EE399830E94E209F02ED0
:1017D000C02E9981D92E8C2D8F19811738F4F601DE
:1017E00061916F018FE70E94E209F5CF64E085E027
:1017F0000E94E20983E00E94DC098093710584E085
:101800000E94DC09809370050E94A62860936C05F5
:1018100070936D0580936E0590936F0569E087E086
:101820000E94E20981E0809373050F90DF91CF91D0
:101830001F910F91FF90DF90CF9008950F931F930A
:101840000E94D70B80917305813099F40E94A628DD
:1018500000916C0510916D0520916E0530916F051A
:10186000601B710B820B930B603A764881409105A7
:1018700048F380917305813031F46EE971E082EEB6
:1018800095E00E94922A1F910F9108950F931F9344
:1018900080917305823021F41092730581E020C09D
:1018A000809173058130D9F40E94A62800916C05BF
:1018B00010916D0520916E0530916F05601B710BC5
:1018C000820B930B613A76488140910540F061E0CC
:1018D00087E00E94E2091092730582E001C080E077
:1018E0001F910F910895CF93DF93EC014AE050E0F0
:1018F0006D2F70E082EE95E00E94602B6EE282EE2A
:1019000095E00E94642ABE0184E0769567958A95E9
:10191000E1F76F7077274AE050E082EE95E00E9491
:10192000602B6EE282EE95E00E94642ABE016F7029
:1019300077274AE050E082EE95E00E94602BDF912D
:10194000CF910895D82FC0E0CD1780F4439A64E674
:1019500070E080E090E00E94C928439864E670E05F
:1019600080E090E00E94C928CF5FEECF6CE271E08A
:1019700080E090E00E94C928E6CF0F931F93CF9399
:10198000DF93EC01062F15E0115051F0CE010E94BB
:101990005B30081741F0602FCE010E946330F4CF16
:1019A00082E00E94A20CDF91CF911F910F910895C8
:1019B000A0E0B0E0EEEDFCE00C94412E482E562E57
:1019C000C0E0D0E0612C712CE12CF12C00E010E0A3
:1019D00041100CC06090D40586E4689E300111244B
:1019E00059E1E52EF12C0AEB15E01EC091E04912F9
:1019F0000FC06090D405E6E46E9E30011124FBE137
:101A00006F0E711C49E2E42EF12C06E715E00CC0C4
:101A100082E0481209C028E1622E77247394EE24F4
:101A2000E394F12C03ED15E043018C0E9D1E109202
:101A30007505109274053401A62CA818B12CC301A9
:101A400001966C01AE14BF04A8F4A00EB11E511093
:101A500006C0C3010E945B30F501808305C0F5011B
:101A60006081C3010E94BD0CF50180810E94610666
:101A70003601E2CFC301511018C0C3010E945B3090
:101A8000B82EC6010E945B302B2D30E0322F22276A
:101A9000282B80917405909175058217930779F42E
:101AA000C0E0D0E05524539493CF36016091750582
:101AB0000E94BD0C60917405C6010E94BD0CC05E01
:101AC000DE4FC13E92E0D90708F482CF852DCDB715
:101AD000DEB7E0E10C945D2E61E082E00E94D80C5C
:101AE000089560E082E00E94D80C8091D305853093
:101AF00020F01092D3050E946C0D8091D305809345
:101B0000D405089561E080E00E94D80C61E081E096
:101B10000E94D80C089560E080E00E94D80C8823D1
:101B200051F060E081E00E94D80C882321F0809180
:101B30007605883349F00E94BF060E947A0681E04C
:101B40000E94DF060E94820D0895882319F06AEA38
:101B500071E002C06EEA71E082EE95E00E94922A86
:101B60000895FF920F931F93CF93DF9369EC7BE06F
:101B700082EE95E00E943E2A40917B0550917C05C3
:101B800060917D0570917E052AE030E082EE95E05F
:101B90000E94672B63EB7BE082EE95E00E943E2A79
:101BA00040917F055091800560918105709182057B
:101BB00020E130E082EE95E00E94672B6DE97BE04A
:101BC00082EE95E00E943E2A4AE050E06091830553
:101BD00082EE95E00E948F2B67E87BE082EE95E035
:101BE0000E943E2A4AE050E06091840582EE95E032
:101BF0000E948F2B61E77BE082EE95E00E943E2AF7
:101C0000C5E8D5E0F12C8E0188818823A9F0FF205A
:101C100031F061EB71E082EE95E00E94612A21963D
:101C20004AE050E0F801608182EE95E00E94582B76
:101C3000F394F8E1FF12E7CF82EE95E00E946C2A60
:101C40006BE57BE082EE95E00E943E2A4AE050E0A0
:101C500060919D0582EE95E00E948F2B66E47BE00B
:101C600082EE95E00E943E2AE0919E05E770F0E04A
:101C7000EE0FFF1FEE57FC4F6081718182EE95E001
:101C80000E94922A61E37BE082EE95E00E943E2A68
:101C900080919E058871883069F028F4811113C005
:101CA00068E27BE00CC0803141F0883161F46CE087
:101CB0007BE005C06CE17BE002C066E17BE082EE88
:101CC00095E00E94802A68EF7AE082EE95E00E941B
:101CD0003E2A409177055091780560917905709181
:101CE0007A052AE030E082EE95E00E94672B6FEDE6
:101CF0007AE082EE95E00E943E2A8091BF058071D5
:101D00000E94A50D66EC7AE082EE95E00E943E2AE4
:101D10008091BF0580740E94A50D6DEA7AE082EE85
:101D200095E00E943E2A8091BF0580720E94A50D19
:101D300060E97AE082EE95E00E943E2A86E795E02F
:101D40000E943708AB01BC012AE030E082EE95E04A
:101D50000E94492B6BE87AE082EE95E00E943E2AD1
:101D600086E795E00E9437089B01AC0160E472E4CD
:101D70008FE090E00E94FE2DBA01A9012AE030E038
:101D800082EE95E00E94492B68E87AE082EE95E0C9
:101D90000E94802ACDB7DEB7E5E00C94682E8F92C2
:101DA0009F92AF92BF92CF92DF92EF92FF928111FA
:101DB00007C06FE77AE082EE95E00E94802A2FC08C
:101DC00090E00E94740724E630E040E050E00E947A
:101DD000FE2DCA01B9012AE030E040E050E00E9447
:101DE000FE2D49015A016B017C012AE030E0B5016A
:101DF000A40182EE95E00E94492B6EE282EE95E00E
:101E00000E94642A2AE030E0B701A60182EE95E044
:101E10000E94492B63E782EE95E00E94A42AFF907E
:101E2000EF90DF90CF90BF90AF909F908F900895EC
:101E30001F93CF93DF9365E77AE082EE95E00E94EF
:101E40003E2A80919F05813041F46CE57AE082EE74
:101E500095E00E94802A10E050C0823019F465E4B9
:101E60007AE0F5CF843019F461E37AE0F0CF853081
:101E700091F766E27AE0EBCFC12FD0E0C930D1050F
:101E80000CF441C068E3610F82EE95E00E94642A81
:101E90006EE17AE082EE95E00E943E2ABE016F5F1D
:101EA0007F4F4AE050E082EE95E00E94282B63E1EC
:101EB0007AE082EE95E00E943E2AC156DA4FE9812F
:101EC000E03218F566E07AE082EE95E00E943E2A64
:101ED0008981803130F06DE673E082EE95E00E94FA
:101EE000612A69816F7070E06F5F7F4F4AE050E058
:101EF00082EE95E00E94312B1F5F809148051817F4
:101F000008F4BACF0FC061E3BECFEF70F0E0EE0F80
:101F1000FF1FEE56FC4F6081718182EE95E00E94BA
:101F2000922AEACF6BEE79E082EE95E00E943E2A9B
:101F30008091B7050E94CF0E60ED79E082EE95E0CA
:101F40000E943E2A8091B8050E94CF0E65EB79E091
:101F500082EE95E00E943E2A8091B9050E94CF0E44
:101F60006AE979E082EE95E00E943E2A4091AF0551
:101F70005091B0056091B1057091B20541155105C0
:101F80006105710539F12AE030E082EE95E00E94AA
:101F9000672B67E679E082EE95E00E943E2A809109
:101FA000B3050E949907AB01BC012AE030E082EE44
:101FB00095E00E94672B63E479E082EE95E00E9451
:101FC0003E2A4AE050E06091B40582EE95E00E941E
:101FD0008F2B06C06AE379E082EE95E00E94802AAA
:101FE0006DE179E082EE95E00E943E2A6091B505B0
:101FF0007091B6054AE050E082EE95E00E94792BA0
:1020000060E079E082EE95E00E943E2A6091AE05A4
:10201000603450F470E06F5F7F4F4AE050E082EE32
:1020200095E00E94312B06C067EF78E082EE95E0E4
:102030000E94802A6AED78E082EE95E00E943E2AB6
:102040008091AD0580FF03C063EB71E002C067EBD8
:1020500071E082EE95E00E94922A6DEB78E082EECC
:1020600095E00E943E2A8091AD0582700E94A50DE8
:102070006EE978E082EE95E00E943E2A8091AD05FF
:1020800084700E94A50D6FE778E082EE95E00E94D3
:102090003E2A8091AD0588700E94A50DDF91CF91F9
:1020A0001F9108950F931F93CF93DF9320914505C0
:1020B0002F3FA9F56FEF75E082EE95E00E943E2A72
:1020C00083E893E00E94730C6EED75E082EE95E07C
:1020D0000E943E2A80914605909147050E94730C0C
:1020E0006BEA75E082EE95E00E94802A68E875E070
:1020F00082EE95E00E94802A60E775E082EE95E02E
:102100000E94802A6BE475E082EE95E00E94802AAE
:1021100082EE95E00E946C2A0E94180F68C0121689
:102120000CF065C0332727FD30958091480590E07D
:10213000821793070CF45BC066E375E082EE95E0CE
:102140000E943E2A60914505772767FD70954AE019
:1021500050E082EE95E00E94312B6BE075E082EE5C
:1021600095E00E943E2A10E008E280914905181788
:10217000D0F5C12FD0E0CC0FDD1FC65BDA4F288130
:1021800030E080914505992787FD909501972817A4
:10219000390739F56BEB71E082EE95E00E94612A18
:1021A0004AE050E0602F82EE95E00E94582B6FEBE2
:1021B00071E082EE95E00E94612AE981EF70F0E023
:1021C000EE0FFF1FEE56FC4F6081718182EE95E0AD
:1021D0000E94612A63EC71E082EE95E00E94612A20
:1021E0000F5F1F5FC2CF82EE95E00E946C2ADF91E5
:1021F000CF911F910F910895FF920F931F93CF934B
:10220000DF93C5E8D5E0F12C8E0188818823D1F1D8
:1022100065EC71E082EE95E00E94612A4AE050E0B0
:102220006F2D82EE95E00E94582B62ED71E082EEF8
:1022300095E00E94612A2196F801208130E0A0E11A
:10224000B7E20E94B82D9B01AC01A0918405B0E0DB
:102250000E94C72DAB01BC0180917B0590917C054C
:10226000A0917D05B0917E05480F591F6A1F7B1F05
:102270002AE030E082EE95E00E94672BF394F8E1CB
:10228000FF12C2CFCDB7DEB7E5E00C94682E1092F6
:10229000DF0485E6E0EEF4E0DF011D928A95E9F7C0
:1022A0000895CF93C82F8F3719F0883009F045C0B3
:1022B000E091DF04EE23D9F1E150E093DF04F0E098
:1022C000E052FB4F10826DE070E082EE95E00E94DC
:1022D0005906C0E08091DF04C81760F4EC2FF0E0ED
:1022E000E052FB4F608170E082EE95E00E9459065B
:1022F000CF5FF0CF60E270E082EE95E00E94590679
:102300006DE070E082EE95E00E945906C0E0809199
:10231000DF04C81778F5EC2FF0E0E052FB4F608146
:1023200070E082EE95E00E945906CF5FF0CF67E043
:1023300082EE95E00E94642A1DC08B3119F40E9440
:1023400047111AC08D30C1F08A30B1F08091DF049E
:10235000843668F76C2F70E082EE95E00E94590693
:10236000E091DF0481E08E0F8093DF04F0E0E05223
:10237000FB4FC08380E001C081E0CF910895CF93EF
:10238000C82F0E94A6286093C8047093C904809344
:10239000CA049093CB04C093DD04CC2329F040E021
:1023A00051EE60E070E004C040E855E260E070E0AB
:1023B00082EE95E00E94EE2CCF9108959091CC048E
:1023C000492F4F7050E0BA016F5F7F4F292F30E0E7
:1023D000E4E035952795EA95E1F76217730759F020
:1023E000FA01E353FB4F808381E0890F8F70907F68
:1023F000892B8093CC0408956EE770E082EE95E01F
:102400000E9459060895A3E1B1E0E9E0F2E10C94DD
:10241000422EE5E8F5E0712C8191882321F0739438
:1024200028E17212F9CF66ED71E082EE95E00E942C
:10243000922A4AE050E0672D82EE95E00E948F2BB1
:1024400080E00E94C10A0E949C0B8E010E5F1F4F0C
:10245000C12CD12C7601C39466246A945C2C0E9412
:102460009A284B015C012091840530E0A0E1B7E29D
:102470000E94B82D9B01AC01C701B6010E94DA2D64
:1024800020917B0530917C0540917D0550917E0522
:10249000620F731F841F951F2091BB053091BC05EF
:1024A0004091BD055091BE052617370748075907CB
:1024B00018F4F801608225C08C2D0E94F50961E0B6
:1024C00070E080E090E00E94C928F80110820E942C
:1024D0009A28681979098A099B09643F7140810526
:1024E000910540F40E940B0AF8019081981778F743
:1024F0008083EDCF50FE03C04298439A02C0429AB7
:1025000043982FEFC21AD20AE20AF20A0F5F1F4F56
:102510008FEFC816D104E104F10409F09FCFCE017A
:102520009395FC01D82E7FEF68EC2E2F281B2715E2
:1025300010F051E056C0DE01129651E02FEF41E05D
:102540003D91321710F0322F01C0452F5F5F5F3F82
:1025500011F0232FF5CF4193242F30E0A1E0B0E01C
:10256000AC0FBD1FA20FB31F5C93413079F0DE01A9
:10257000A20FB31F5C93423049F0AFEFBFEFAC0F37
:10258000BD1FA20FB31F6C934E3F78F6A2E0B0E0E0
:10259000AC0FBD1FA20FB31F7C934D3F30F6A3E0DD
:1025A000B0E0AC0FBD1FA20FB31F6C93BECF452F81
:1025B000242F30E0FC01E20FF31F6081AFEFB0E0A9
:1025C000AC0FBD1FA20FB31F2C91621748F44150EE
:1025D000DC01A40FB11D2C9120836C934111E8CF35
:1025E0005F5F571520F3372D369520E0231770F4E1
:1025F000DC01A20FB11D4C91522F530FFC01E50FCE
:10260000F11D50815C9340832E5FF0CFF5E8EF2EF3
:10261000F5E0FF2E8C01802F8D19871598F4F801B5
:10262000C1908F014AE050E06C2D82EE95E00E944F
:10263000582B6CE282EE95E00E94642AF701C19269
:102640007F01E9CF82EE95E00E946C2A81E0CD5EA9
:10265000DE4FEFE00C945E2E1F920F920FB60F929A
:1026600011241F932F933F934F935F936F937F9307
:102670008F939F93AF93BF93CF93DF93EF93FF938A
:10268000C0918600D0918700809187049091880442
:102690002091A904211155C09E01281B390B80915E
:1026A000BF059091C005A091C105B091C20585FDFF
:1026B00002C036952795253C49E03407B8F1409192
:1026C0000A0150E060E070E02CE1B695A79597957F
:1026D00087952A95D1F70097A105B10521F481E0EE
:1026E00090E0A0E0B0E084179507A607B707D8F4FC
:1026F00080910A018F3FB9F040E080910A014817AC
:1027000080F4842F90E0880F991FFC01E757FB4F5E
:1027100020813181FC01E55FFE4F318320834F5FD3
:10272000ECCF1092AA0410920A010BC02D3B82E05C
:10273000380720F080910A018031D8F08FEF809324
:102740000A01D0938804C0938704FF91EF91DF9131
:10275000CF91BF91AF919F918F917F916F915F9139
:102760004F913F912F911F910F900FBE0F901F908F
:10277000189510910A0181E0810F80930A01C90127
:102780000E942109E12FF0E0EE0FFF1FE757FB4FFA
:1027900091838083D6CF83E0809380008AE9809301
:1027A00081008091BF0586FD05C080918100806415
:1027B000809381008FEF9FEF909389008093880032
:1027C00080916F00806280936F0008950E94710D68
:1027D0008091D405843011F41092D40508956F309F
:1027E00018F086958058089589E0689F802D1124FF
:1027F0000895A0E0B0E0EFEFF3E10C94492EC82F6C
:102800000E94A628009138041091390420913A04BE
:1028100030913B046B017C01C01AD10AE20AF30A31
:102820009701860149E8C41643E1D406E104F104A6
:1028300010F010923C046093380470933904809334
:102840003A0490933B042091A9048FEF820F8230C9
:10285000D8F5E0913C04EE2309F44EC1E13011F4C7
:1028600082E0B8C1E03108F034C181E08E0F80937E
:102870003C04F0E0E757FB4FC083803109F0ACC166
:10288000EBE8F4E0213029F4A181A695A69580819A
:1028900008C080819181A92FA695A695A6959695A9
:1028A0008795A03148F4B0E090E0AA0FBB1FA55F68
:1028B000BE4F11969C938E931092AA04329684E098
:1028C000E939F807F9F688C1233009F005C1E0912C
:1028D0003C04E11104C0CF3009F07EC10DC1E831E4
:1028E00048F481E08E0F80933C04F0E0E857FB4F02
:1028F000C08372C1E83109F0ECC0C111EAC040E008
:1029000050E0ABE0CA01B3E0880F991FBA95E1F738
:10291000A49F9001A59F300D1124F901E757FB4FAB
:102920006081E1817E2F777075956795FC01EE0FD0
:10293000FF1FE55FFE4F71836083F901E657FB4F90
:10294000B081B695B695B695E181FE2FF295FF0F51
:10295000F07E6F2F6B2BE695E695E6957E2F7770D0
:1029600075956795FC01EE0FFF1FE35FFE4F7183C6
:102970006083F901E557FB4FB081B295B695B695E6
:10298000B370C181DC2FDD0FDD0F6D2F6B2BC29576
:10299000C695C695C370E281E170EE0FEE0F7E2FF3
:1029A0007C2B75956795FC01EE0FFF1FE15FFE4FD5
:1029B00071836083F901E357FB4FB081B695E181E4
:1029C000FE2FF795FF27F7956F2F6B2BE6957E2F40
:1029D000777075956795FC01EE0FFF1FEF5EFE4F58
:1029E00071836083F901E257FB4FB081B295BF70EC
:1029F000E181FE2FF295F07F6F2F6B2BE295EF7048
:102A00007E2F777075956795FC01EE0FFF1FED5EC9
:102A1000FE4F71836083F901E157FB4FB081BB1F0B
:102A2000BB27BB1FC181DC2FDD0F6D2F6B2BCC1F94
:102A3000CC27CC1FE281E370EE0F7E2F7C2B7595A7
:102A40006795FC01EE0FFF1FEB5EFE4F7183608305
:102A5000F901EF56FB4FB081B695B695E181FE2F97
:102A6000F295FF0FFF0FF07C6F2F6B2BE695E6952D
:102A70007E2F777075956795FC01EE0FFF1FE95E5D
:102A8000FE4F71836083F901EE56FB4F2081229542
:102A9000269527703181E32FEE0FEE0FEE0F6E2F8C
:102AA000622B732F72957695777075956795FC01FB
:102AB000EE0FFF1FE75EFE4F718360834F5F5F4F36
:102AC0004230510509F01ECF80919F0483FF109280
:102AD000AA0410923C0480C0243009F07DC06091AB
:102AE0003C0461110BC0C83AB1F410927505109204
:102AF000740588EA0E94610681E06CC0613019F4B7
:102B0000C093370404C0623031F4C09336048C2F74
:102B10000E9461065AC0E09136042E2F30E0220F49
:102B2000331F462F50E0C9010296841795073CF0E9
:102B3000633268F7FA01EA57FB4FC083E8CF2D5F95
:102B40003F4F8C2F90E0609174057091750542178E
:102B5000530749F4982F8827862797279093750560
:102B60008093740532C06817790769F5809137043E
:102B7000813049F5E13118F080E180933604F0901E
:102B80003604CAE8D4E000E010E00F15D0F4FE01EE
:102B90003197808190E0982F88272881822B63E0ED
:102BA000969587956A95E1F70E942109F801EE0F45
:102BB000FF1FE55FFE4F918380830F5F1F4F2296BB
:102BC000E4CF1092AA0410923C0480913C04882324
:102BD00019F08F5F80933C04CDB7DEB7E8E00C942A
:102BE000652EE82FF0E0E654FA4FE185E03150F42D
:102BF000F894F0E0EE0FFF1FE55FFE4F80819181BA
:102C000078940895E03121F0E13131F483E101C09D
:102C100082E10E94E829089580E092E00895A2E20E
:102C2000B0E0E5E1F6E10C943F2E9E012F5F3F4FAF
:102C300080E1D9011D928A95E9F764E072E082EEA5
:102C400095E029A33AA30E94922A0E94BF0B1D8AF5
:102C50001E8A1F8A188E312C212C00E0812C912C89
:102C60005401412C74E7572E7BE8672E72E3772ED0
:102C7000E0E5CE2EE3ECDE2EE12CF12C84EF91E0AA
:102C8000A0E0B0E08D8F9E8FAF8FB8A380E09EEC68
:102C9000ADEEB4E3898F9A8FAB8FBC8F80E094E761
:102CA000ABE8B2E3898B9A8BAB8BBC8B82EE95E061
:102CB0000E94A62B892B09F4E1C082EE95E00E94C8
:102CC000D32B9C0133272C32310509F442C0ACF4DC
:102CD0002332310509F0ABC019821A821B821C8293
:102CE0001D821E821F82188619861A861B861C86E4
:102CF0001D861E861F86188A60C02434310529F07F
:102D00002335310509F4B2C092C064E482EE95E047
:102D10000E94642A2AE030E040E054E76BE872E366
:102D200082EE95E00E94F22A6CE282EE95E00E942B
:102D3000642A2AE030E040E05EEC6DEE74E382EE5F
:102D400095E00E94F22A6CE282EE95E00E94A42AAD
:102D5000ADCF0F5F043009F0A9CF29813A814B81B3
:102D60005C81A8EEB3E00E94C72D698B7A8B8B8BB8
:102D70009C8B2D813E814F8158850E94C72D698F84
:102D80007A8F8B8F9C8F29853A854B855C852D8F1B
:102D90003E8F4F8F58A32D853E854F8558890E94C1
:102DA000C72D6B017C0160323EE4730781059105FC
:102DB00030F462E38CE10E94E20900E077CF6033F7
:102DC00045E774078105910510F462E2F3CF6034A2
:102DD0005CE975078105910510F466E2EBCF80E5AB
:102DE000C81683ECD806E104F10410F462E1E2CFE6
:102DF00090E6C9169AEED906E104F10410F465E1F3
:102E0000D9CFA0E7CA16A1E1DA06A1E0EA06F104EB
:102E100010F461E0CFCFB0EACB16B6E8DB06B1E044
:102E2000EB06F10410F463E0C5CF65E0C3CF10ED0D
:102E3000180F1A3008F03ACFE1E0F0E0EC0FFD1F78
:102E400024E0029FE00DF11D112420813181428197
:102E50005381AAE0B0E00E94C72D610F711D811D52
:102E6000911D608371838283938320CF49885A8820
:102E70006B887C88812C912C540118CF811491048B
:102E8000A104B10489F4C301B2010E94510A61E0B6
:102E900070E080E090E00E94C9281D8A1E8A1F8A87
:102EA000188E312C22242A948D8D9E8DAF8DB8A141
:102EB00088169906AA06BB06D0F40E940B0A2D8933
:102EC0003E894F89588D280F311D411D511D2D8B75
:102ED0003E8B4F8B588F381608F4382E821508F425
:102EE000282E3FEF831A930AA30AB30A56C0C301E0
:102EF000B20128EE33E040E050E00E94FE2DBA011E
:102F0000A9012AE030E082EE95E00E94492B6CE2B4
:102F100082EE95E00E94642A4AE050E0632D82EE42
:102F200095E00E94582B6CE282EE95E00E94642AA4
:102F30006D897E898F89988DA50194010E94FE2D4F
:102F4000BA01A9012AE030E082EE95E00E94492B07
:102F50006CE282EE95E00E94642A4AE050E0622D25
:102F600082EE95E00E94582B6CE282EE95E00E9482
:102F7000A42A4C0C5D1C6E1C7F1C898D9A8DAB8D18
:102F8000BC8D84159505A605B70520F449885A8897
:102F90006B887C88812C912C540129893A894B8932
:102FA0005C89283E33404105510509F07FCEA29649
:102FB000E2E10C945B2EACE1B0E0E1EEF7E10C94C1
:102FC000492E0E94A6286B017C0181E00E94C10A63
:102FD00014E703E0198361E0CE0101960E941E0C04
:102FE000009373050E949C0B6AEF70E080E090E014
:102FF0000E94C92880917305833089F482EE95E0A0
:103000000E94A62B892B59F40E94A6286C197D09D1
:103010008E099F096038734C894C9140D8F2809199
:103020007305833009F44FC08FE70E94BA090E94EC
:10303000CD098983843511F083E05CC00E94CD09FD
:1030400010924605809347050E94CD0920914605C0
:1030500030914705280F311D3093470520934605D1
:103060000E94CD09809348050E94CD0980934905AF
:10307000813110F7F12C0F2D10E08091490590E07F
:10308000880F991F0817190740F40E94CD09F8010D
:10309000E65BFA4F8083F394EECF80E7898361E0AB
:1030A000CE0101960E941E0C83E0809373050E945E
:1030B0009C0B62E370E080E090E00E94C928809160
:1030C0007305833011F482E015C08FE70E94BA09BE
:1030D0000E94CD098983803509F0AECF0FE915E054
:1030E0000E94CD09F80181938F01F5E00A3B1F078B
:1030F000B9F781E06C96E8E00C94652E8091450567
:10310000992787FD9095A92FB92FFC013196EB30B7
:10311000F10508F066C0EC5CFF4F0C94762E62E778
:1031200078E082EE95E00E94802A83E893E00E9496
:10313000730C6AE578E082EE95E00E94802A65E3F0
:1031400078E082EE95E00E94802A6BE078E082EEE3
:1031500095E00E94802A6AEE77E082EE95E00E9478
:10316000802A6DEB77E082EE95E00E94802A67E985
:1031700077E082EE95E00E94802A63E777E082EEB6
:1031800095E00E94802A6CE477E082EE95E00E9450
:10319000802A82EE95E00E946C2A0E94B10D21C027
:1031A0006FE277E01AC06AE077E017C065EF76E07B
:1031B00014C066ED76E011C062E976E00EC06DE7FE
:1031C00076E00BC068E676E082EE95E00E94802A09
:1031D00062E276E002C06CE076E082EE95E00E946A
:1031E000802A6AE070E080E090E00E94C92882EEC8
:1031F00095E00E94A62B892B29F082EE95E00E9493
:10320000D32BF5CF0895ACE1B0E0E9E0F9E10C94FF
:10321000492E909145059F3F09F023C1482F50E06A
:10322000FA013A97EF36F10508F00FC1E15CFF4F64
:103230000C94762E61E172E0A0C06DE172E082EE46
:1032400095E00E94922A85E789838BE1EFE9F5E01A
:10325000DE01129601900D928A95E1F76CE1CE01A4
:1032600001960E941E0C0E949C0B83E080937305C4
:1032700068EC70E080E090E00E94C92880917305BE
:10328000843009F0E2C08FE70E94BA090E94CD099C
:103290008983853509F0D9C06DEE74E082EE95E042
:1032A0000E94802A6FEC74E082EE95E00E94802AF2
:1032B00061EB74E096C065E372E082EE95E00E94F7
:1032C000922A89E6898361E0CE0101960E941E0C54
:1032D0000E949C0B83E08093730568EC70E080E0B3
:1032E00090E00E94C92880917305843009F0ADC038
:1032F0008FE70E94BA090E94CD0989838E010E5F73
:103300001F4F7E014DE1E40EF11C0E94CD09F80132
:1033100081938F01EE15FF05C1F78BE1FE01329617
:10332000AFE9B5E001900D928A95E1F78981893482
:1033300009F08BC063E974E082EE95E00E94802A78
:1033400065E774E082EE95E00E94802A67E574E00C
:1033500048C06FE472E082EE95E00E94922A8EEF00
:103360008093450572C080528750805390914805E4
:10337000981708F066C06EE572E082EE95E00E9454
:10338000922A63C084E18093450560E274E029C01D
:1033900085E18093450569EE73E023C086E1809363
:1033A000450562EB73E01DC087E18093450568E643
:1033B00073E017C088E18093450567E573E011C0AD
:1033C00089E18093450563E473E00BC08AE1809353
:1033D00045056EE273E005C08BE18093450566E02C
:1033E00073E082EE95E00E94802A2FC06CEE72E0BE
:1033F00082EE95E00E94802A8091AD0591E01DC08B
:1034000066ED72E082EE95E00E94802A8091AD0523
:1034100092E013C061EC72E082EE95E00E94802A97
:103420008091AD0594E009C066EA72E082EE95E015
:103430000E94802A8091AD0598E089278093AD0590
:103440008FEF809345050E94521082EE95E00E9416
:10345000A62B892B09F45AC182EE95E00E94D32B4A
:10346000F4CF0E945111882309F450C18091DF04E8
:10347000811104C08FEF8093450540C140E050E0CA
:1034800060E070E080EE94E00E94ED2E40914505F2
:10349000042F112707FD1095212F312FF8013197A7
:1034A000EB31F10508F01AC1E255FF4F0C94762E6E
:1034B000552747FD50952091480530E024173507E2
:1034C0000CF40CC18B019C01015011092109310937
:1034D000003211052105310558F0C0904905EBE493
:1034E000F5E0F12CD12CA8E2EA2E415051090FC091
:1034F000FA01E156FA4F61506083D8C0DF0111979D
:103500002C9130E02417350729F0F3943296FC1003
:10351000F5CFCAC00E2D10E020E030E006171707E7
:103520002807390741F42081DA01A156BA4F1196D4
:103530002C93DD24D394E394E8CF6F3F710581058C
:10354000910511F008F0CAC06093B705AFC06F3F96
:1035500071058105910511F008F0C0C06093B805B0
:10356000A5C06F3F71058105910511F008F0B6C047
:103570006093B9059BC02091E00420622037E9F4F4
:1035800040E050E060E070E081EE94E00E94ED2EBB
:103590009B01AC01DC01CB010197A109B10908979E
:1035A000A105B10508F0ADC0A4EDB0E30E94C72DA0
:1035B0006A5E7C4A8A46954E24C02636E9F440E08D
:1035C00050E060E070E081EE94E00E94ED2E9B01FF
:1035D000AC01DC01CB010197A109B1090797A10555
:1035E000B10508F08EC0A8EAB1E60E94C72D645E5E
:1035F0007C438E46944E05C0611571058105910589
:1036000071F08B019C0114572B4832430130FAE5CD
:103610001F07F2E62F07F2E03F0708F05FC0609354
:10362000AF057093B0058093B1059093B2053EC08D
:103630006F3F71058105910511F008F04FC060934F
:10364000B30534C08B019C010150110921093109D6
:103650000F3F11052105310508F040C06093B40506
:1036600025C08B019C01045C1940210931090D34EE
:103670004DE114072105310528F47093B6056093D8
:10368000B50514C0611571058105910521F48FEF11
:103690008093AE050BC06134710581059105F0F48E
:1036A00061506093AE0502C0DD20C1F08091DE0460
:1036B00081111AC080917F0590918005A0918105AC
:1036C000B09182050196A11DB11D80937F05909355
:1036D0008005A0938105B093820506C060E772E083
:1036E00082EE95E00E94922A0E9447118FEF80930C
:1036F00045056AE082EE95E00E94A42A0E945210DD
:1037000005C061E070E080E090E07BCF6C96E8E07F
:103710000C94652E6AE572E082EE95E00E94802AA4
:1037200062E472E082EE95E00E94802A82EE95E0EB
:103730000E94A62B892B31F082EE95E00E94D32BBC
:103740000E9403190E94DB17823029F0833051F464
:103750006DE072E002C064E272E082EE95E00E94E9
:10376000802A08958FEF809345051092DE040E9411
:103770005210809145058E3F69F082EE95E00E94DF
:10378000A62B892BB1F382EE95E00E94D32B0E94E9
:103790000319EFCF08950F931F93109145051F3F15
:1037A00009F0D2C0893409F457C000F5883309F410
:1037B00069C058F4803309F477C008F061C08B31D8
:1037C00009F440C08132B1F1B9C0813409F487C035
:1037D00030F4893309F466C0803461F1AFC08234BB
:1037E00009F48EC0863409F448C0A8C0823609F4B2
:1037F00087C078F4883531F128F48235C1F18335FA
:10380000E1F09CC08A3509F494C0813609F467C0A0
:1038100095C0823761F128F4863679F18936E1F076
:103820008DC0883779F08A3709F483C0833709F06F
:1038300085C003C061E172E015C00E94820D6EE890
:1038400072E004C00E948B0D68EA72E082EE95E09F
:103850000E94922A8EEF70C00E947A060E94BF06D4
:1038600067EC72E082EE95E00E94922A67C081E0E8
:103870000E94DF0660EE72E0F5CF0E94FC105EC091
:1038800080535AC06AEF71E082EE95E00E94802A70
:1038900090919E0588E0890F8871977E892B80938F
:1038A0009E051AC089E048C067EE71E082EE95E09F
:1038B0000E94802A8091BF059091C005A091C1050A
:1038C000B091C20520E182278093BF059093C00587
:1038D000A093C105B093C205109345052FC061EDBB
:1038E00071E082EE95E00E94802A8091BF05909160
:1038F000C005A091C105B091C20540E4842710C065
:1039000060EC71E082EE95E00E94802A8091BF0514
:103910009091C005A091C105B091C20520E2822717
:103920008093BF059093C005A093C105B093C205D5
:1039300002C00E948A1B8FEF809345058091450548
:103940008E3F09F0D4C0DDC00E945111882309F4D4
:10395000D8C08091DF04811104C08FEF80934505AA
:10396000C6C040E050E060E070E080EE94E00E946D
:10397000ED2E00914505112707FD1095212F312FC0
:10398000F8013197E930F10508F0B4C0E753FF4F73
:103990000C94762E8B019C01015014472B48324326
:1039A0000F3F19452246324008F0A4C060937B05C2
:1039B00070937C0580937D0590937E0577C060931E
:1039C0007F0570938005809381059093820581E047
:1039D0008093DE046BC0683071058105910508F0A5
:1039E00089C06093830562C08B019C01015011095D
:1039F000210931090A3011052105310508F07AC085
:103A00006093840553C061EB71E080EE94E00E9406
:103A1000273010E0009799F00E940130009779F06C
:103A2000183130F4E12FF0E0EA58FA4F87871F5F32
:103A300061EB71E080E090E00E942730EBCF18311D
:103A4000A8F5E12FF0E0EA58FA4F17861F5FF7CF8D
:103A5000653071058105910508F04CC060939D05A6
:103A600025C08B019C010150110921093109063043
:103A7000110521053105F0F520919E05287F262BA3
:103A800020939E0513C08B019C010150110921094F
:103A900031090115124C2140310560F5609377051D
:103AA000709378058093790590937A058091DE0470
:103AB000811113C080917F0590918005A0918105AF
:103AC000B09182050196A11DB11D80937F05909351
:103AD0008005A0938105B09382050E9447118FEF66
:103AE000809345056AE082EE95E00E94A42A0E9438
:103AF0007E1807C060E772E082EE95E00E94922A8D
:103B0000ECCF1F910F9108958FEF80934505109290
:103B1000DE040E947E18809145058E3F69F082EE9A
:103B200095E00E94A62B892BB1F382EE95E00E94CE
:103B3000D32B0E94CB1BEFCF6AE070E080E090E0D7
:103B40000E94C92882EE95E00E94A62B892B29F0BD
:103B500082EE95E00E94D32BF5CF0895CF93C82F26
:103B6000682F82EE95E00E94002C90916A059C27B8
:103B700090936A05CF910895A1E0B0E0E2ECFDE1F9
:103B80000C944F2E99830E94AE1D9981892F0E941B
:103B9000AE1D2196E2E00C946B2E1F93CF93DF9322
:103BA000182FEB0110926A0565EB70E082EE95E04C
:103BB0000E94590662E670E082EE95E00E94590686
:103BC000812F0E94AE1DCE010E94BC1DDF91CF91BE
:103BD0001F91089560916A0582EE95E00E94002C85
:103BE0000895A1E2B0E0E7EFFDE10C944B2E7B01DC
:103BF0008A018C3009F453C108F040C0863009F4C2
:103C0000BCC018F5833009F491C070F4813009F418
:103C100072C0823009F048C26BE170E082E00E941D
:103C2000CD1D0FE915E078C0843009F487C08530D8
:103C300009F03AC26091490570E0660F771F85E090
:103C40000E94CD1D0AE415E086C0893009F4A7C0A2
:103C500070F4873009F49BC0883009F025C261E018
:103C600070E088E00E94CD1D8091D40523C28A3087
:103C700009F4CAC08B3009F4F2C016C28A3609F4BE
:103C800075C1D8F4873609F43AC138F4853609F499
:103C90000EC1863609F41FC107C2883609F437C140
:103CA000893609F001C261E070E089E60E94CD1D0D
:103CB0000E947A060E94BF06F5C18D3609F4D4C170
:103CC00038F48B3609F491C18C3609F49AC1ECC1F1
:103CD0008E3609F4DCC1873C09F0E6C161E070E092
:103CE00087EC0E94CD1D81E00E94AE1D0E94EA1D5E
:103CF00010926B05E3C169E270E081E00E94CD1D86
:103D000006E715E0F80181918F010E94AE1DF5E0F4
:103D10000F391F07B9F7D0C1F80181918F010E94B7
:103D2000AE1DF5E00A3B1F07B9F7C6C161E070E0C0
:103D300083E00E94CD1D0E94DB17BCC161E070E0F2
:103D400084E00E94CD1D81E00E94AE1D0E94EA1D0C
:103D50000E940F16B3C18091490590E0880F991F0A
:103D600098012A5435402817390708F0A5C1F801F1
:103D700081918F010E94AE1DEECF62E070E086E07F
:103D80000E94CD1D83E893E00E94BC1D95C161E0B7
:103D900070E087E00E94CD1D809148058BC186E6CA
:103DA000898361E0CE0101960E941E0C0E949C0B4B
:103DB00083E08093730568EC70E080E090E00E94FF
:103DC000C928809173058430D9F48FE70E94BA091D
:103DD0000E94CD098983863469F460E270E089E04D
:103DE0000E94CD1D10E20E94CD090E94AE1D11500F
:103DF000D1F762C161E070E089E00E94CD1D52C13F
:103E000061E070E089E053C169E170E08AE00E94FE
:103E1000CD1D81E08093BA05209172058091BF0588
:103E20009091C005A091C105B091C205222311F067
:103E3000806801C08F778093BF059093C005A093E1
:103E4000C105B093C2050AEB15E0F80181918F011D
:103E50000E94AE1DF5E0033D1F07B9F72DC161E2D9
:103E600070E08BE00E94CD1D8091AA048F3F39F055
:103E70008091AA0491E0980F9093AA0402C08091C7
:103E8000AA040E94AE1D10E0812F0E94F1150E942D
:103E90004C090E94BC1D1F5F1031B1F70DC161E0DC
:103EA00070E08CE00E94CD1D8091D30503C161E0DC
:103EB00070E085E60E94CD1D89E2E816F10409F064
:103EC000F8C0D801E6E7F5E08D91819385E0EF3900
:103ED000F807D1F7E7C061E070E086E60E94CD1DEB
:103EE000EBE1EE16F10409F0E4C0D801EFE9F5E0EA
:103EF0008D91819385E0EA3BF807D1F7D3C061E06B
:103F000070E087E60E94CD1D0E94820DCBC061E06B
:103F100070E088E60E94CD1D85E789838BE1EFE99B
:103F2000F5E0DE01129601900D928A95E1F76CE1C1
:103F3000CE0101960E941E0C0E949C0B83E0809390
:103F4000730560E273E080E090E00E94C9288091F0
:103F50007305843009F0ADC08FE70E94BA090E9452
:103F6000CD098983853509F0A4C09CC061E070E06B
:103F70008AE60E94CD1D89E6898361E0CE01019623
:103F80000E941E0C0E949C0B83E08093730560E2EC
:103F900073E080E090E00E94C9288091730584302E
:103FA00009F087C08FE70E94BA090E94CD09898372
:103FB0008E010E5F1F4F7E01EDE1EE0EF11C0E949F
:103FC000CD09F80181938F01EE15FF05C1F78BE153
:103FD000FE013296AFE9B5E001900D928A95E1F7C6
:103FE0008981893409F065C05DC061E070E08BE6CD
:103FF0000E94CD1DF80180818093D4050E948B0D15
:1040000051C061E070E08CE60E94CD1DF0E2EF1639
:10401000F10461F487E6898380E2F801DE011296FB
:1040200001900D928A95E1F761E203C087E48983EC
:1040300061E0CE0101960E941E0C0E949C0B83E061
:10404000809373056CE474E080E090E00E94C928DE
:1040500080917305843069F58FE70E94BA090E9448
:10406000CD09873431F51EC061E070E08DE60E9415
:10407000CD1D89E1E816F104E1F4D801EAEBF5E0A1
:104080008D91819385E0E33DF807D1F70BC061E0A6
:1040900070E08EE60E94CD1DF80180818093D305EB
:1040A0000E946C0D81E006C061E070E08AEC0E9425
:1040B000CD1D80E00E94AE1D0E94EA1DA196E6E0A3
:1040C0000C94672EA0E0B0E0E8E6F0E20C94492EF4
:1040D000CAECD3E014E606E035E0F32E44E0E42E2B
:1040E00053E0D52E62E0C62E82EE95E00E94A62B0C
:1040F000892B09F49BC082EE95E00E94D32B282FD8
:10410000809335044091340450E04730510560F706
:10411000FA01EE52FF4F0C94762E853B29F781E091
:1041200080933404E1CF823609F07DC0C09234041C
:10413000DBCF8093330480933204D0923404D4CF05
:104140009C01332730933104209330049091320442
:10415000982790933204E0923404C6CF382F222758
:104160004091300450913104242B352B309331048D
:104170002093300490913204982790933204F09267
:1041800034042536310508F4AFCF61E070E08CECE3
:104190000E94CD1D81E00E94AE1D0E94EA1D43C019
:1041A00020912E0430912F04F901E653FC4F8083B7
:1041B00090913204982790933204C901019690930C
:1041C0002F0480932E042091300430913104821703
:1041D000930708F489CF0093340486CF809132048A
:1041E00082130BC060912E0470912F044AEC53E0AF
:1041F000809133040E94F11D0DC062E070E08BECF1
:104200000E94CD1D809133040E94AE1D80916A05ED
:104210000E94AE1DFE01812F11928A95E9F710923E
:104220002F0410922E04109234045ECFCDB7DEB767
:10423000E8E00C94652E81E080936B0580916B051E
:10424000882349F082EE95E00E94A62B892BB1F3DA
:104250000E946220F3CF0895AAE2B0E0E2E3F1E227
:104260000C94472E0E949A286B017C0181E00E94E9
:10427000C10A82EE95E00E94A62B892B29F082EEDE
:1042800095E00E94D32BF5CF439811E072E6B72E4C
:10429000E9E2AE2E03E00E949A286C197D098E098E
:1042A0009F09693C710581059105D0F11123C1F188
:1042B0000E949A286B017C01429A80ED97E00E944F
:1042C000B607B982E6E7F5E0DE0112968A2D019085
:1042D0000D928A95E1F76AE2CE0101960E941E0CCA
:1042E000429880E090E00E94B607009373050E9418
:1042F0009C0B62E370E080E090E00E94C92880910E
:104300007305843061F4009373058FE70E94BA0946
:104310000E94CD0911E0823419F410E001C011E0CF
:1043200082E10E94BF29892B81F411E00EC0439ADB
:10433000429A82EE95E00E94D32B8D309105A9F030
:104340005CF40A9791F04398429882EE95E00E94BF
:10435000A62B892B61F79FCF8332910579F08234A8
:10436000910589F70E941B21EECF62EB71E082EE8E
:1043700095E00E94802A0E94841DE5CF0E940F16BE
:10438000E2CF8F929F92AF92BF92CF92DF92EF9245
:10439000FF921F93CF93DF9382E10E94BF29892B65
:1043A00009F089C068EC70E080E090E00E94C928C4
:1043B00080E090E00E94B6070E949A284B015C01C1
:1043C0006B017C0180ECC80E82E1D81EE11CF11C5F
:1043D0000E949A286C157D058E059F0530F482E1B8
:1043E0000E94BF29892BA1F364C082E10E94BF29EA
:1043F000892B09F05EC080ED97E00E94B6070E940D
:104400009A286B017C01D0E0C1E088E4880E86E246
:10441000981EA11CB11C11E082E10E94BF29892BCA
:1044200021F58C149D04AE04BF0430F480ED97E0B8
:104430000E94B607D1E0F0CF0E949A286C197D093E
:104440008E099F09693C71058105910528F30E9439
:104450009A286B017C01C12719F080ED97E002C01A
:1044600080E090E00E94B607D7CF80E090E00E9405
:10447000B607DD23B9F08091D30590E0019665E0A1
:1044800070E00E94EA2D8093D3050E946C0D0E947B
:10449000E6130E948B0D64EF71E080E090E00E94D3
:1044A000C92809C080E00E94DF060E9403120E9412
:1044B000820D0E942C21DF91CF911F91FF90EF90F0
:1044C000DF90CF90BF90AF909F908F900895CF9244
:1044D000DF92EF92FF9280E00E941D080E94F40795
:1044E00061E081E10E94532961E080E10E9453294B
:1044F00060E082E10E94532960E088E00E94532935
:1045000061E088E00E948C290E949F0740E052EC05
:1045100061E070E082EE95E00E94EE2C0E94E613CE
:104520000E948B0D0E94CB138FEF8093AA040E94F0
:10453000090878940E949A286B017C018091AA0452
:104540008F3F59F40E949A286C197D098E099F09A2
:10455000603D77408105910588F380ED97E00E94EA
:10456000B60761E082E10E948C29439A82EE95E0D1
:104570000E94A62B892B29F082EE95E00E94D32B76
:10458000F5CF6DEF72E082EE95E00E94612A83E83C
:1045900093E00E94730C64E173E082EE95E00E9468
:1045A000612A4AE050E068E070E082EE95E00E9407
:1045B000312B62E370E080E090E00E94C92882EE37
:1045C00095E00E94A62B04970CF182EE95E00E94E4
:1045D000D32B82349105D1F482EE95E00E94D32B47
:1045E0008E34910599F482EE95E00E94D32B8434A9
:1045F000910561F482EE95E00E94D32B819731F40E
:1046000080E090E00E94B6070E942C21409177053F
:10461000509178056091790570917A05DB01CA01A6
:104620000197A109B1090497A105B10568F4409368
:10463000A904433029F440EA56E861E070E004C080
:1046400040E052EC61E070E082EE95E00E94EE2CDA
:104650000E94C121439880E090E00E94B6070E942A
:10466000CB131092C5048091BF0583FF11C08091C8
:104670008B05882351F080919205882331F0809139
:104680009905882311F087E001C085E08093C50477
:1046900080E00E94C10A8091C6040E94F5090E9430
:1046A0009C0B10923F0410923E0410923D04F12C9A
:1046B0008091D4058F15B0F062E370E080E090E067
:1046C0000E94C92880ED97E00E94B60762E370E07F
:1046D00080E090E00E94C92880E090E00E94B60748
:1046E000F394E6CF80919E0584FF08C0982F9871BF
:1046F00081E0983109F080E00E94BF118FE00E94B4
:104700001D08FF90EF90DF90CF900895EF92FF92F9
:104710000F931F93CF93DF938C016EE770E082EECF
:1047200095E00E945906E801F12CF0E2EF2E8E018F
:1047300088818D57823048F46DE770E082EE95E015
:104740000E94590688818E2588832196F801608110
:1047500082EE95E00E94002CF394F9E0FF12E7CF7F
:104760006EE770E082EE95E00E945906CDB7DEB7A5
:10477000E6E00C94672EA9E0B0E0E1ECF3E20C94E3
:104780004F2E9091C70491110EC09EEF99838A839A
:104790006B8350E0559547954C832D831986188679
:1047A0001F821E822EC04091CC04842F90E0B4E082
:1047B00095958795BA95E1F7242F2F7030E08217F1
:1047C000930719F18DEF89831B82FE01349650E027
:1047D000842F90E0A4E095958795AA95E1F7242F82
:1047E0002F7030E08217930749F0DC01A353BB4FD1
:1047F0008C918193405F5F5F563051F74093CC04BA
:104800005A83CE0101960E9486238091C70490E0CE
:10481000019666E070E00E94EA2D8093C704299615
:10482000E2E00C946B2EA0E0B0E0E9E1F4E20C943D
:10483000482E6C016EE770E082EE95E00E9459060A
:104840008601E12CF12CC0E0D0E030E2B32EF8017B
:10485000608183E8860F823078F46DE770E082EE45
:1048600095E00E945906F80160816B2570E082EEA8
:1048700095E00E94590604C082EE95E00E94002C4B
:10488000E114F10459F0F80180819E01280F311DD7
:10489000C901C92FDD27C80FD91FDD273FEFE31A54
:1048A000F30A89E0E816F10459F028E0E216F10471
:1048B00021F48C2F8095F60180870F5F1F4FC7CFA3
:1048C000CDB7DEB7E9E00C94642EA9E0B0E0EBE6EA
:1048D000F4E20C944F2EE82F362F8091C70490E01D
:1048E000019664E270E00E94EA2D8093C70458E9C3
:1048F000598350E15A83813089F048F08230B9F011
:104900008330D9F48B8381EF8C833D8319C085E09C
:104910008B8381EF8C832F5F2D8312C08B8381EF7C
:104920008C8384E6489FA00111245D8309C084E044
:104930008B8381EF8C83ED8303C00E94FC1104C044
:10494000CE0101960E9413242996E2E00C946B2E6E
:10495000A2E0B0E0EEEAF4E20C94442E182F762E9A
:104960002A8349830E94A6286B017C018091DD0483
:104970008090C8049090C904A090CA04B090CB0461
:104980002A8149818823C1F0D701C6018819990974
:10499000AA09BB094C015D0191EE89169EE29906B8
:1049A000A104B10420F1241708F4422F202F672D11
:1049B000812F0E94652413C0D701C6018819990967
:1049C000AA09BB094C015D0191E3891695E7990697
:1049D000A104B10460F0672D812F0E94BB23C09217
:1049E000C804D092C904E092CA04F092CB04229683
:1049F000EDE00C94602EA2E2B0E0E1E0F5E20C9470
:104A0000452E8CE00E94DC0981110DC06CE173E041
:104A100082EE95E00E94922A439A80E00E94C10AA9
:104A20000E949C0B439882EE95E00E94A62B892B56
:104A300001F182EE95E00E94D32B9091A904992375
:104A400019F00E94F913EFCF40913E0450E09A0113
:104A50002F5F3F4F2F71332760913F0470E026177F
:104A6000370709F3FA01E75BFB4F808320933E048D
:104A7000DACF80917305843009F086C00E94A628A1
:104A8000611571058105910549F06093B704709334
:104A9000B8048093B9049093BA040CC081E090E00C
:104AA000A0E0B0E08093B7049093B804A093B90459
:104AB000B093BA048091AD049091AE04816090935C
:104AC000AE048093AD0483E0809373058FE70E946A
:104AD000BA0909E614E00E94CD09F80181938F011B
:104AE000F4E002371F07B9F720917204809169043E
:104AF000982F922796FF3BC090E4922790937204E0
:104B0000982F98739833F1F410E0212F30E08091C2
:104B10006904877090E0821793074CF11F5F209122
:104B20009E05812F90E0FC01E759FB4F24FF04C054
:104B300080810E94DE11E9CF608182EE95E00E94C3
:104B4000002CE3CF8F7399F480916A048093B604AC
:104B500080916B048093B40480916C048093B304BF
:104B600080916F0490E09093AC048093AB048091AB
:104B70003D04813019F482E080933D0480913D042E
:104B8000833011F410923D040E94A6286B017C0131
:104B90008091AF049091B004A091B104B091B2049F
:104BA0000097A105B105C9F0A7019601281B390B93
:104BB0004A0B5B0BDA01C901883B9B40A105B1059B
:104BC00060F00E940B0A8093B5041092AF0410921B
:104BD000B0041092B1041092B2048091BB04909181
:104BE000BC04A091BD04B091BE0446015701881ACF
:104BF000990AAA0ABB0A86E795E00E94370886163A
:104C00009706A806B90608F4A8C0C092BB04D092C3
:104C1000BC04E092BD04F092BE040E94570680914D
:104C2000AA048830A0F08091BF059091C005A091A2
:104C3000C105B091C2055CE1B695A795979587959A
:104C40005A95D1F7892B8A2B8B2B09F09EC1809125
:104C5000AA048F5F8093AA048091B7049091B8044E
:104C6000A091B904B091BA040097A105B105F1F083
:104C7000C81AD90AEA0AFB0A86E795E00E943708B3
:104C80006C157D058E059F0508F006C18091BF0556
:104C900084FD04C080ED97E00E94B6071092B7042F
:104CA0001092B8041092B9041092BA049091720450
:104CB000907C9093720450913E0480913F04209127
:104CC0003D04581709F405C1223009F002C190587B
:104CD00090937204E0919E05E770F0E0E658FC4F77
:104CE0006081693008F0DDC0615040E04613DBC0F0
:104CF00080933F0487E3840F90917204892B809303
:104D000072044093400483E080933D04429A809172
:104D100083059091C504911129C10E94BC0A80911C
:104D2000C6040E94F509E0919E05E770F0E0E658A0
:104D3000FC4F608182E794E00E94D70BE091C604AB
:104D4000EF5FE093C604E83109F41CC1F0E0EA58D3
:104D5000FA4F8785882309F415C10E94460C8130DB
:104D600069F580919E05887149F18091AD0490911B
:104D7000AE04880F991F9093AE048093AD0483E036
:104D8000809373050E949C0B0E94A6286093AF0439
:104D90007093B0048093B1049093B204672B682B96
:104DA000692B61F481E090E0A0E0B0E08093AF0473
:104DB0009093B004A093B104B093B20480919E0587
:104DC00084FF1FC08091AD049091AE048E7F0E943D
:104DD0006D09182F6091AB048091B6040E94EF1307
:104DE000482F612F8091B50449A30E94EF130091D1
:104DF000D405282F49A16091B3048091B4040E9486
:104E0000A82442988091C3048130C1F018F0823008
:104E1000B1F1C8C082E10E94BF29892B09F0C2C04C
:104E200081E08093C3040E949A286093BF0470932A
:104E3000C0048093C1049093C204B4C082E10E9474
:104E4000BF29892B31F50E949A28C090BF04D090C9
:104E5000C004E090C104F090C2046C197D098E0971
:104E60009F09693E73408105910508F49BC082E06B
:104E70008093C30480ED97E00E94B60793C082E15F
:104E80000E94BF29892B09F48DC080E090E00E9428
:104E9000B6071092C30486C080E090E00E94B60777
:104EA00005CF68E022CF851709F422CF4F5F242F6A
:104EB00030E090E0F901EE58FB4FDC01A75BBB4FFF
:104EC0007C917083F901E05CFB4F708301968F71D8
:104ED0000DCF2430B1F42091400481E494E0A3E7A5
:104EE000B4E0FC013E2F381B321718F431913D938A
:104EF000F9CF87E3820F90917204892B809372041B
:104F000002CF8091C304823051F491609093720477
:104F1000439A8E010F5F1F4FF12CB80110C04398C8
:104F200080913D04811103C081E080933D04809114
:104F30003D04833071F784E080933D04EACF8F2DE8
:104F400069A37AA30E94F115F801819391938F01CF
:104F5000F39469A17AA1F0E1FF12F1CF80919E054F
:104F600043E754E087700E94BC08D0CE882309F440
:104F7000D4CE2091C40431E0320F3093C4042913FD
:104F8000CCCE0CC01092C604E8CE8091AA04883022
:104F900009F4439A89E08093AA04DFCE1092C404F6
:104FA0008150BBCEA296ECE00C94612E8230E8F4E6
:104FB000E82FF0E0EE0FFF1FEB52FA4F7183608392
:104FC000813041F0809169008C7F842B809369004F
:104FD000E89A089580916900440F551F440F551FAA
:104FE000837F842B80936900E99A08951F920F9222
:104FF0000FB60F9211242F933F934F935F936F93AC
:105000007F938F939F93AF93BF93EF93FF93809181
:10501000D5059091D605892B29F0E091D505F09121
:10502000D6050995FF91EF91BF91AF919F918F9117
:105030007F916F915F914F913F912F910F900FBE94
:105040000F901F9018951F920F920FB60F92112478
:105050002F933F934F935F936F937F938F939F9380
:10506000AF93BF93EF93FF938091D7059091D805AD
:10507000892B29F0E091D705F091D8050995FF918A
:10508000EF91BF91AF919F918F917F916F915F91C0
:105090004F913F912F910F900FBE0F901F90189539
:1050A0001F920F920FB60F9211242F933F938F935D
:1050B0009F93AF93BF938091DA059091DB05A09108
:1050C000DC05B091DD053091D90523E0230F2D37A4
:1050D00020F40196A11DB11D05C026E8230F0296FC
:1050E000A11DB11D2093D9058093DA059093DB05AE
:1050F000A093DC05B093DD058091DE059091DF057E
:10510000A091E005B091E1050196A11DB11D80932C
:10511000DE059093DF05A093E005B093E105BF9114
:10512000AF919F918F913F912F910F900FBE0F9054
:105130001F9018952FB7F8946091DA057091DB05F0
:105140008091DC059091DD052FBF08953FB7F8945D
:105150008091DE059091DF05A091E005B091E10519
:1051600026B5A89B05C02F3F19F00196A11DB11DC2
:105170003FBF6627782F892F9A2F620F711D811DDF
:10518000911D42E0660F771F881F991F4A95D1F73E
:105190000895CF92DF92EF92FF92CF93DF936B014E
:1051A0007C010E94A628EB01C114D104E104F104A2
:1051B00079F00E94A6286C1B7D0B683E7340A0F31B
:1051C00081E0C81AD108E108F108C851DC4FECCFE2
:1051D000DF91CF91FF90EF90DF90CF90089578947A
:1051E00084B5826084BD84B5816084BD85B58260EC
:1051F00085BD85B5816085BDEEE6F0E0808181608A
:105200008083E1E8F0E01082808182608083808189
:1052100081608083E0E8F0E0808181608083E1EB61
:10522000F0E0808184608083E0EBF0E08081816049
:105230008083EAE7F0E080818460808380818260FF
:1052400080838081816080838081806880831092E8
:10525000C1000895833081F028F4813099F08230C4
:10526000A1F008958630A9F08730B9F08430D1F4E8
:10527000809180008F7D03C0809180008F77809324
:105280008000089584B58F7702C084B58F7D84BD7A
:1052900008958091B0008F7703C08091B0008F7D1A
:1052A0008093B0000895CF93DF9390E0FC01ED5020
:1052B000F44F2491FC01E95FF34F8491882349F175
:1052C00090E0880F991FFC01E15DF34FA591B49127
:1052D0008B5D934FFC01C591D4919FB7611108C0BC
:1052E000F8948C91209582238C93888182230AC024
:1052F000623051F4F8948C91322F309583238C9343
:105300008881822B888304C0F8948C91822B8C93A3
:105310009FBFDF91CF910895A1E0B0E0E2E9F9E20B
:105320000C944D2E282F30E0F901E152F44F849176
:10533000F901ED50F44F1491F901E95FF34F049135
:105340000023C9F0882321F069830E942A296981FA
:10535000E02FF0E0EE0FFF1FEB5DF34FA591B4914E
:105360009FB7F8948C91611103C01095812301C0FF
:10537000812B8C939FBF2196E4E00C94692ECF93F0
:10538000DF93282F30E0F901E152F44F8491F901C5
:10539000ED50F44FD491F901E95FF34FC491CC2360
:1053A00091F081110E942A29EC2FF0E0EE0FFF1FEF
:1053B000E55EF34FA591B4912C912D2381E090E00F
:1053C00021F480E002C080E090E0DF91CF91089569
:1053D0008E3008F08E50877020919D0190E4299FB7
:1053E00090011124822B80937C0080917A0080644C
:1053F00080937A0080917A0086FDFCCF80917800BE
:105400002091790090E0922B0895A0E0B0E0EBE0CD
:10541000FAE20C94492E6C017A01EB01E60EF71EBC
:1054200000E010E0CE15DF0561F06991D601ED9145
:10543000FC910190F081E02DC6010995080F191F1C
:10544000F1CFC801CDB7DEB7E8E00C94652E611549
:10545000710589F0DB010D900020E9F7AD014150A5
:105460005109461B570BDC01ED91FC910280F38141
:10547000E02D0995089580E090E00895EF92FF9265
:105480000F931F93CF93DF938C01FB01C0E0D0E01B
:1054900064917F018FEFE81AF80A662361F0D80162
:1054A000ED91FC910190F081E02DC8010995C80FA4
:1054B000D91FF701EDCFCE01CDB7DEB7E6E00C94F2
:1054C000672E0E94272A0895DC01ED91FC9101903E
:1054D000F081E02D099508950F931F93CF93DF93EB
:1054E000EC016DE00E94642A8C016AE0CE010E940A
:1054F000642A800F911FDF91CF911F910F91089522
:105500000F931F93CF93DF93EC010E943E2A8C01EF
:10551000CE010E946C2A800F911FDF91CF911F91C5
:105520000F9108950F931F93CF93DF93EC010E9487
:10553000272A8C01CE010E946C2A800F911FDF91D7
:10554000CF911F910F9108950F931F93CF93DF93E6
:10555000EC010E94642A8C01CE010E946C2A800F0B
:10556000911FDF91CF911F910F910895A1E2B0E0BB
:10557000ECEBFAE20C94452E7C01C42EE52FCB0116
:10558000D22E19A221E02D1510F02AE0D22E8E0184
:105590000F5D1F4F8D2C912CA12CB12C6C2D7E2FCB
:1055A000A50194010E94FE2D8C2DD29E80191124FC
:1055B000015011098A3010F4805D01C0895CF80146
:1055C0008083211531054105510521F0C22EE32FBD
:1055D000CA01E4CFB801C7010E94272AA196ECE0D6
:1055E0000C94612EA0E0B0E0E8EFFAE20C94492EB2
:1055F000EC016A017B012115310541F4E881F98153
:105600000190F081E02D642F09951DC02A303105ED
:10561000A9F477FF12C06DE20E94642A8C0144272E
:105620005527BA014C195D096E097F092AE0CE01A0
:105630000E94B62A800F911F06C02AE0B701A6017A
:10564000CE010E94B62ACDB7DEB7E8E00C94652EF5
:105650009A01AB01662757FD6095762F0E94F22ACA
:1056600008950F931F93CF93DF93EC019A01AB0141
:10567000662757FD6095762F0E94F22A8C01CE0195
:105680000E946C2A800F911FDF91CF911F910F9183
:1056900008952115310549F4DC01ED91FC9101904B
:1056A000F081E02D642F099508950E94B62A08958F
:1056B0009A01462F50E060E070E00E94492B089567
:1056C0009A01AB0160E070E00E94492B08950F93AE
:1056D0001F93CF93DF93EC010E94492B8C01CE01E5
:1056E0000E946C2A800F911FDF91CF911F910F9123
:1056F00008950F931F93CF93DF93EC019A01AB01B1
:1057000060E070E00E94492B8C01CE010E946C2A5F
:10571000800F911FDF91CF911F910F9108950F93EB
:105720001F93CF93DF93EC019A01462F50E060E086
:1057300070E00E94492B8C01CE010E946C2A800FE0
:10574000911FDF91CF911F910F910895FC01248546
:105750003585F901E05CFF4F80819181F901EE5BB5
:10576000FF4F20813181821B930B8F7399270895FE
:10577000FC0184859585FC01E05CFF4F40815181EF
:10578000FC01EE5BFF4F208131814217530741F04E
:105790000190F081E02DE80FF91F808190E00895DD
:1057A0008FEF9FEF0895FC0184859585FC01E05CF7
:1057B000FF4F40815181FC01EE5BFF4F2081318121
:1057C0004217530779F0A081B181A80FB91F8C91BE
:1057D000208131812F5F3F4F2F7333273183208307
:1057E00090E008958FEF9FEF0895FC0181A1882339
:1057F00029F0A489B5898C9186FFFBCF11A2089569
:10580000CF93DF93FC0126853785D901A05CBF4F7C
:105810008D919C91119701968F739927E901CE5B29
:10582000DF4F4881598184179507D9F30D90BC91BA
:10583000A02DA20FB31F6C93A685B785A05CBF4FA8
:1058400011969C938E93A689B7892C9181E090E064
:10585000078C02C0880F991F0A94E2F7282B2C931B
:1058600081E081A30488F589E02D808180648083B4
:1058700081E090E0DF91CF91089508951F920F92FB
:105880000FB60F9211242F933F934F938F939F93B3
:10589000EF93FF938091C00082FD1CC04091C60031
:1058A000809188069091890601968F73992720919F
:1058B0008A0630918B068217930771F0E091880673
:1058C000F0918906E85BF94F4083909389068093B5
:1058D000880602C08091C600FF91EF919F918F9141
:1058E0004F913F912F910F900FBE0F901F901895E1
:1058F00082EE95E00E94A62B892B11F00E943D2C90
:1059000008951F920F920FB60F9211242F933F9379
:105910008F939F93EF93FF93209144063091450618
:1059200080914606909147062817390731F48091F7
:10593000C1008F7D8093C10014C0E0914606F091B4
:105940004706EC5FF94F208180914606909147060B
:1059500001968F739927909347068093460620936C
:10596000C600FF91EF919F918F913F912F910F90E2
:105970000FBE0F901F901895A0E0B0E0E2ECFCE2A3
:105980000C94452EFC011382128288EE93E0A0E075
:10599000B0E084839583A683B7838CEB93E09183F7
:1059A00080837587648757874687318B208B138B5D
:1059B000028BF58AE48AD78AC68AB18EA08E938E2E
:1059C000828E8F85848F8889858F8989868F8A8941
:1059D000878F8B8980A3ECE00C94612ECF92DF92AD
:1059E000EF92FF92CF93DF93EC016A017B014115A7
:1059F00081EE580761057105F9F0EC89FD8981E0B8
:105A000090E008A002C0880F991F0A94E2F78083F3
:105A100060E079E08DE390E0A70196010E94FE2D01
:105A200021503109410951095695479537952795D8
:105A3000211580E1380798F0EC89FD89108260E833
:105A400074E88EE190E0A70196010E94FE2D21509E
:105A50003109410951095695479537952795E889A8
:105A6000F9893083EA89FB89208319A2EE89FF89AD
:105A7000408181E090E09C010C8C02C0220F331F1A
:105A80000A94E2F7422B4083EE89FF8940819C0112
:105A90000D8C02C0220F331F0A94E2F7422B408381
:105AA000EE89FF8940819C010E8C02C0220F331FBA
:105AB0000A94E2F7422B4083EE89FF8920810F8C04
:105AC00002C0880F991F0A94E2F780958223808391
:105AD000DF91CF91FF90EF90DF90CF9008958F925C
:105AE0009F92AF92BF92CF92DF92EF92FF920F936D
:105AF0001F9381E08F9385E08F9387E08F9383E0FE
:105B00008F9384E08F93E6EC8E2E912CF2ECAF2EE7
:105B1000B12CA1ECCA2ED12CB0ECEB2EF12C04EC64
:105B200010E025EC30E044E056E068E476E082EEF8
:105B300095E00E94BC2C0F900F900F900F900F904B
:105B40001F910F91FF90EF90DF90CF90BF90AF909B
:105B50009F908F9008950E94EF280E946722C8E7C7
:105B6000DCE20E94FB242097E1F30E94782CF9CF1D
:105B7000A29FB001B39FC001A39F700D811D11248E
:105B8000911DB29F700D811D1124911D08950E94D9
:105B9000B82DA59F900DB49F900DA49F800D911DD1
:105BA00011240895B7FF0C94C72D0E94C72D821BA6
:105BB000930B0895DB018F939F930E94C72DBF9194
:105BC000AF91A29F800D911DA39F900DB29F900D4C
:105BD0001124089597FB072E16F4009407D077FD43
:105BE00009D00E947C2E07FC05D03EF4909581954B
:105BF0009F4F0895709561957F4F0895A1E21A2EE9
:105C0000AA1BBB1BFD010DC0AA1FBB1FEE1FFF1F60
:105C1000A217B307E407F50720F0A21BB30BE40BB0
:105C2000F50B661F771F881F991F1A9469F76095F7
:105C30007095809590959B01AC01BD01CF010895B1
:105C4000052E97FB1EF400940E94372E57FD07D0B7
:105C50000E94FE2D07FC03D04EF40C94372E509575
:105C60004095309521953F4F4F4F5F4F0895909548
:105C70008095709561957F4F8F4F9F4F08952F921C
:105C80003F924F925F926F927F928F929F92AF92CC
:105C9000BF92CF92DF92EF92FF920F931F93CF9319
:105CA000DF93CDB7DEB7CA1BDB0B0FB6F894DEBFB0
:105CB0000FBECDBF09942A88398848885F846E84D6
:105CC0007D848C849B84AA84B984C884DF80EE8020
:105CD000FD800C811B81AA81B981CE0FD11D0FB629
:105CE000F894DEBF0FBECDBFED010895EE0FFF1F8C
:105CF0000590F491E02D0994AA1BBB1B51E107C04C
:105D0000AA1FBB1FA617B70710F0A61BB70B881F4B
:105D1000991F5A95A9F780959095BC01CD010895DA
:105D20008F929F92AF92BF92CF92DF92EF92FF92AB
:105D3000CF93DF93EC01688179818A819B81611522
:105D400071058105910521F464E279ED8BE597E019
:105D50002DE133EF41E050E00E94202E49015A012D
:105D60009B01AC01A7EAB1E40E94C72D6B017C0145
:105D7000ACEEB4EFA50194010E94D52DC60ED71E3E
:105D8000E81EF91EF7FE06C081E0C81AD108E10836
:105D900080E8F80AC882D982EA82FB82C701B6018C
:105DA0009F77DF91CF91FF90EF90DF90CF90BF90E2
:105DB000AF909F908F9008950E94902E089586E056
:105DC00091E00E94902E0895609306017093070160
:105DD000809308019093090108952F923F925F925A
:105DE0006F927F928F929F92AF92BF92CF92DF92EB
:105DF000EF92FF920F931F93CF93DF938B01EA01F2
:105E00006115710521F0DB018C9311969C9320970D
:105E100039F09E01225031092332310508F0D8C0F3
:105E20007C016701BFEFCB1ADB0A5601F7016080E6
:105E3000862D90E00E941F30892B11F07601F1CF62
:105E4000FDE26F120AC0570182E0A80EB11CD70113
:105E500011966C90772473940BC0BBE26B1207C051
:105E60005701E2E0AE0EB11CD70111966C90712C77
:105E7000CE018F7E892B89F4B0E36B1237C0F50118
:105E800080818F7D8835D1F46180F2E0AF0EB11C46
:105E9000872D8260782EC0E1D0E0CA30D10551F163
:105EA000C031D10521F0C830D10599F409C0CC2406
:105EB000CA94DC2CEC2CAFE0FA2E22C0209769F7B4
:105EC000C8E0D0E0CC24CA94DC2CEC2CFFE1FF2EFF
:105ED00017C06FEF7FEFCB019E01442737FD409540
:105EE000542F0E94FE2D69017A010AC02097A9F65D
:105EF000CAE0D0E0E9E9CE2EDC2CEC2CE9E1FE2E64
:105F0000F50160E020E030E0A9014E01AA2497FCF1
:105F1000A094BA2C1F0170ED572E560CA9E0A515C0
:105F200070F48FEB860D8A3118F499EC592E06C067
:105F30008FE9860D8A3148F589EA582E560C852D51
:105F400090E08C179D070CF56F3FD9F0C216D30671
:105F5000E406F50698F0C501B4010E94DA2D9B0114
:105F6000AC01852D90E0A0E0B0E0280F391F4A1F5A
:105F70005B1F281739074A075B0710F46FEF01C052
:105F800061E03196D1016C90C5CF0115110551F03A
:105F9000662311F0319703C071FE04C03297D80117
:105FA000ED93FC9370FE07C0509540953095219578
:105FB0003F4F4F4F5F4F67FF10C082E290E09093DA
:105FC0008D0680938C066FEF7FEF8FEF9FEF07C0FA
:105FD00060E070E080E090E002C0B901CA01DF91AA
:105FE000CF911F910F91FF90EF90DF90CF90BF90D6
:105FF000AF909F908F907F906F905F903F902F9089
:106000000895FC0188279927E89421912032E9F32B
:10601000293010F02E30C8F32B3241F02D3239F4F4
:10602000689404C00E945330820F911D2191205327
:106030002A30C0F31EF4909581959F4F08959111D9
:1060400050C0803219F089508550D0F7089548EC3F
:1060500053E00E942C300895FA01A191B08100977D
:1060600019F41097E1F0CD01DC01CD010D90002075
:1060700011F4C00113C0FB012191222319F0201556
:10608000D9F7F3CFFB012191201519F41E92119637
:1060900006C02223C1F70D900020A1F7D001FA011C
:1060A000A193B08308957AE0979F902D879F802DCC
:1060B000910D11240895F999FECF92BD81BDF89AF2
:1060C000992780B50895262FF999FECF1FBA92BD62
:1060D00081BD20BD0FB6F894FA9AF99A0FBE0196C9
:0C60E0000895992788270895F894FFCFB1
:1060EC0000008E06200001000000FF0002000200EC
:1060FC000200020002000200020002000200020084
:10610C0002000200020002000200028025000005CD
:10611C00400AA1204EA50020244EA52C2330C012ED
:10612C0000001A400AA1204EA5001B1E27522C234A
:10613C00308025000005400AA1204EA50020244EE9
:10614C00A52C2330004B000006400AD0009D4900CE
:10615C007B289D492C233000E1000005400A4501B5
:10616C00D7DC03B81E0EBF00232E48E801008A407E
:10617C000A6001555502AD1E20000023C801545879
:10618C002074696D656F75742100596573004E6FCD
:10619C00002C00386368004E2F41002C205B005D02
:1061AC002028002900486F70206368616E6E656C52
:1061BC00200020402000456E746572696E67206176
:1061CC0064617074697665206368616E6E656C20BD
:1061DC0073656C656374696F6E2C207069636B6991
:1061EC006E673A007363616E6E6572206D6F6465E5
:1061FC00004E4F5420454E41424C45440053656E71
:10620C0064696E672073657474696E677320746F4C
:10621C002052580A00526573657474696E67207356
:10622C00657474696E6773206F6E2052580A004152
:10623C00626F727465642065646974730A00696EB8
:10624C0076616C69642073656C656374696F6E004C
:10625C000D0A496E76616C696420696E70757420E4
:10626C002D20646973636172646564210700536552
:10627C007474696E677320736176656420746F2023
:10628C00454550524F4D0A005265766572746564EF
:10629C002073657474696E67732066726F6D204528
:1062AC004550524F4D0A004C6F6164656420666125
:1062BC0063746F72792064656661756C74730A001F
:1062CC004B657920616E64206368616E6E656C73DA
:1062DC002072616E646F6D697A65640A004F706537
:1062EC006E4C52536E6720545820737461727469EB
:1062FC006E672000206F6E20485720006D6F64750C
:10630C006C65206C6F636B65643F00342B34003814
:10631C0000382B340031320031322B34003136004E
:10632C0050504D0052535349005344410053434C79
:10633C0000525844005458440041494E004C4245C8
:10634C0045500053504B54524D005342555300533B
:10635C00554D44004C4C494E440000070B0C101199
:10636C001500B7012B032F033103350338033D030D
:10637C00B7014003440349034D035103550359032B
:10638C005D0363036A036F0374038D028D028D0238
:10639C008D02160A1322312900000000002C052A58
:0863AC00A62BD32BB82BF52B17
:00000001FF
